:100000000C9477000C945C0D0C94890D0C949F005B
:100010000C949F000C949F000C949F000C949F00E4
:100020000C949F000C949F000C949F000C949F00D4
:100030000C949F000C949F000C949F000C949F00C4
:100040000C94B60D0C94AC000C948F0F0C94DD0F37
:100050000C949F000C949F000C949F000C949F00A4
:100060000C94CB0A0C949F00486F6C6964617944CE
:1000700075696E6F30352D313600486F6C6964617B
:10008000794475696E6F30352D31360000000000FF
:10009000240027002A0000000000250028002B0073
:1000A00000000000230026002900040404040404C6
:1000B0000404020202020202030303030303010217
:1000C00004081020408001020408102001020408E6
:1000D00010200000000700020100000304060000D9
:1000E000000000000000390142091D0D49111124D2
:1000F0001FBECFEFD8E0DEBFCDBF11E0A0E0B1E082
:10010000E8E1FAE202C005900D92AA34B107D9F7EE
:1001100016E0AAE4B1E001C01D92A933B107E1F7EE
:1001200010E0CEEED0E004C02297FE010E94FA1348
:10013000C63ED107C9F70E949F110C940A150C9472
:100140000000FC01A081B1812D913C91F90109953C
:10015000089581E0089508951F920F920FB60F92AF
:1001600011242F933F934F935F936F938F939F939C
:10017000EF93FF936EB58091710490E04091090177
:1001800050910A019A01220F331F240F351F821745
:10019000930774F480917104E0913804F09139046C
:1001A000E80FF11D6083809171048F5F809371046B
:1001B000FF91EF919F918F916F915F914F913F913F
:1001C0002F910F900FBE0F901F901895FC01549A1D
:1001D00080E182838BE290E0948383830895DF93B0
:1001E000CF9300D00F92CDB7DEB7DC01AB01ED911C
:1001F000FC910680F781E02D19821A821B82BE01D4
:100200006F5F7F4F20E009950F900F900F90CF9177
:10021000DF9108956BB900140014001427FF4BB947
:1002200000140014001400144BB90014001400143E
:1002300008950F936BB900140014001427FF4BB9F5
:1002400000140014001400144BB9001402E00A95C5
:10025000F1F70F9108956BB900140014001426FFF4
:100260004BB900140014001400144BB9001400140E
:10027000089508950E94FE0D60930F017093100180
:10028000809311019093120108951F9380910901A9
:1002900090910A01892B09F443C082E00E945E0F0D
:1002A000892B49F4809172048823D1F5109271044E
:1002B00088E060E033C08091710490E040910901D2
:1002C00050910A019A01220F331F240F351F821704
:1002D000930724F480913C048823E1F011E010930B
:1002E0003A040E94FE0D2091630430916404442777
:1002F00037FD4095542F260F371F481F591F209355
:100300006D0430936E0440936F0450937004109307
:10031000720406C01092710488E061E00E942B0F05
:100320001F9108958EE480937C0062E070E080E08D
:1003300090E00E94320E80917A00806480937A006F
:1003400080917A0086FDFCCF8091780090E0A0E05B
:10035000B0E060917900362F20E0442737FD4095CA
:10036000542F282B392B4A2B5B2B60E070E381E163
:1003700090E00E94C913CA01B90108950F931F9319
:100380008C018DEB94E060E570E00E94D708612F4E
:10039000772767FD7A958DEB94E00E948A091070AB
:1003A0008DEB94E0602F0E948A098DEB94E00E940F
:1003B000CD098DEB94E060E570E041E050E00E94F3
:1003C000DE098DEB94E00E94E108892B11F480E0B6
:1003D00004C08DEB94E00E94EA081F910F910895EC
:1003E000DF92EF92FF920F931F938C01D62E8DEB2D
:1003F000E82E84E0F82EC70160E570E00E94D7087F
:10040000612F772767FD7A95C7010E948A091070CE
:10041000C701602F0E948A09C7016D2D0E948A09B9
:10042000C7010E94CD0965E070E080E090E00E9485
:10043000320E1F910F91FF90EF90DF9008950F9370
:100440001F93CF93DF93182F8F3339F483E196E016
:1004500068E670E00E94261293C18B3519F08D3545
:1004600081F407C08DEB94E068E070E00E94010A1F
:1004700004C08DEB94E00E94E20983E196E0612FD5
:100480007DC1813491F4809167048370825F60E064
:100490000E94BF0E8091670483700E949D0E809120
:1004A000670483700E949D0EC2C0823479F585E096
:1004B0000E945E0F8C0186E00E945E0F892B19F06E
:1004C000C0E0D0E002C0C2E0D0E087E00E945E0F52
:1004D000892B19F020E030E002C024E030E060E039
:1004E00070E0012B11F461E070E080913E049927E7
:1004F00087FD909544E0880F991F4A95E1F7682B96
:10050000792B6C2B7D2B622B732B2CC18334F9F44C
:100510008091650490916604029771F460910B01DB
:1005200070910C0180916704909168040E9494136B
:10053000609169040E94F00160910B0170910C01BF
:1005400080916704909168040E9494131FC08434C2
:1005500039F580913D0490E0209165043091660466
:1005600082239323892B81F0609167047091680442
:100570008091410490914204681779070CF060E083
:1005800085E090E00E94F00185E090E00E94BE01CD
:10059000682F83E196E04AE050E00E94E112F0C04B
:1005A0008534B1F48091650490916604892B59F0EB
:1005B00010923B048091670490916804892B19F094
:1005C00081E080933B0460E070E080913B04A4C034
:1005D000873469F4809167048370825F61E00E94D0
:1005E000BF0E809167048370825F60E00EC0883424
:1005F00079F4809167048370825F61E00E94BF0E8E
:10060000809167048370825F61E00E942B0F09C0B4
:10061000893479F4809167048370825F60E00E947E
:10062000BF0E809167048370825F0E945E0FBC01E1
:1006300099C08C3401F58091650490916604892BF2
:10064000A9F080913D04882389F06091670470913E
:1006500068046B3F710514F06AEF70E070930A0153
:100660006093090183E090E00E94F001609109012C
:1006700070910A0177C0803599F48091650490915A
:100680006604892B41F080916704909168049093EF
:10069000400480933F0460913F047091400462C025
:1006A000823519F58091650490916604029781F472
:1006B000E0916704F0916804EF70F070EE0FFF1F97
:1006C000ED5BFB4F8091690490916A049183808374
:1006D000E0916704F0916804EF70F070EE0FFF1F77
:1006E000ED5BFB4F608171813DC08435D1F4809119
:1006F000650490916604892B59F010923C04809116
:10070000670490916804892B19F081E080933C0480
:1007100060E070E080913C04882321F161E070E0AA
:1007200021C0863559F40E949201AB01BC0183E1DE
:1007300096E02AE030E00E943F1322C08735C9F4DA
:100740008091650490916604892B41F08091670443
:1007500090916804909364048093630460916304AF
:100760007091640483E196E04AE050E00E945313E4
:1007700007C080322CF083E196E06FE30E943A12CA
:10078000DF91CF911F910F9108950F931F93CF93F6
:10079000DF9383E196E040E052EC61E070E00E947C
:1007A000181085E062E00E94BF0E86E062E00E94C1
:1007B000BF0E87E062E00E94BF0E88E061E00E9409
:1007C000BF0E88E061E00E942B0F8CE061E00E9488
:1007D000BF0E8CB580648CBDC0910901D0910A0117
:1007E0001C161D06D4F4009138011091390189E0DE
:1007F00090E00E94AE11FC011582168217821086CD
:1008000088E191E091838083C801BF014AE451E00F
:100810009E0100E010E00E947A0C8AE491E090933F
:10082000390480933804109271041092720480E0AD
:1008300065E471E041E050E00E94390D81E06AE337
:1008400071E042E050E00E94390D8CB580688CBDAB
:1008500085E00E945E0F892B29F480913E048F5F12
:1008600080933E0486E00E945E0F892B29F48091DC
:100870003E048E5F80933E0487E00E945E0F892BCA
:1008800029F480913E048C5F80933E048DEB94E0CC
:100890000E94E20980E090E00E94BE01883669F57E
:1008A00081E090E00E94BE01813039F580933D04E3
:1008B00082E090E00E94BE0190E0880F991F880FAF
:1008C000991F90930C0180930B0183E090E00E94AC
:1008D000BE018093090110920A0184E090E00E9419
:1008E000BE01809341041092420485E090E00E9492
:1008F000BE0180933F041092400483E196E06AE7D2
:1009000070E00E942612DF91CF911F910F91089500
:100910000F931F938C010E940C0E9B01AC01F801F8
:1009200080819181A281B381281B390B4A0B5B0B1B
:10093000223331054105510534F482E390E0821BF6
:10094000930B0E94580E1F910F9108954F925F9242
:100950007F928F929F92AF92BF92CF92DF92EF924F
:10096000FF920F931F93CF93DF932C01162F072F26
:100970004A01722E05960E948804F894212F302F88
:10098000C901EC015401AA0CBB1CA80CB91CA80E8F
:10099000B91ECBB020E1C22AEBB03FEEE322EBB8A8
:1009A0000981272D029F012D90C015E08BE290E078
:1009B0006C2D4E2D202F0E940A01000F1150B1F70F
:1009C00000148BE290E06C2D4E2D202F0E94190117
:1009D0008BE290E06C2D4E2D202F0E942B01F88091
:1009E0003F2D272D329F312DF32ECBB8001400144C
:1009F000001405FFEBB80014001400140014EBB849
:100A000002E00A95F1F715E08BE290E06C2D4E2D97
:100A10002F2D0E940A01FF0C1150B1F700148BE238
:100A200090E06C2D4E2D2F2D0E9419018BE290E04D
:100A30006C2D4E2D2F2D0E942B01DA803D2D272D60
:100A4000329F312DD32ECBB8001400140014F5FEC4
:100A5000EBB80014001400140014EBB802E00A957F
:100A6000F1F715E08BE290E06C2D4E2D2D2D0E94BC
:100A70000A01DD0C1150B1F70014CBB800140014BA
:100A80000014D7FEEBB80014001400140014EBB8E7
:100A90000014001400140014001423968BE290E05C
:100AA0006C2D4E2D2D2D0E942B010981372D039F7A
:100AB000012DCBB8001400140014D5FEEBB80014BF
:100AC000001400140014EBB80014CA15DB0508F478
:100AD0006CCF1124E0908605F09087050091880581
:100AE00010918905B401E3E0660F771FEA95E1F7FD
:100AF000680D791D882777FD8095982F28EE33E0C3
:100B000040E050E00E94C913E20EF31E041F151FBF
:100B1000E0928605F0928705009388051093890579
:100B200078940E940C0EF201658376838783908708
:100B3000DF91CF911F910F91FF90EF90DF90CF90B9
:100B4000BF90AF909F908F907F905F904F9008954F
:100B50002F923F925F926F927F928F929F92AF926D
:100B6000BF92CF92DF92EF92FF920F931F93DF938A
:100B7000CF9300D000D0CDB7DEB71C017C836B8350
:100B80004A01522E05960E948804F8945401AA0C3A
:100B9000BB1CA80CB91C2B813C81A20EB31ECBB090
:100BA00030E1C32AEBB08FEEE822EBB8EB81FC8199
:100BB0003196FA83E983EB81FC811181252D129F07
:100BC000112D3F0199C005E08BE290E06C2D4E2D78
:100BD000212F0E940A01110F0150B1F700148BE27E
:100BE00090E06C2D4E2D212F0E9419018BE290E098
:100BF0006C2D4E2D212F0E942B01EB81FC81F0806A
:100C00002F2D352D239F212DF22ECBB8001400144B
:100C1000001415FFEBB80014001400140014EBB816
:100C200002E00A95F1F705E08BE290E06C2D4E2D85
:100C30002F2D0E940A01FF0C0150B1F700148BE226
:100C400090E06C2D4E2D2F2D0E9419018BE290E02B
:100C50006C2D4E2D2F2D0E942B01EB81FC81D2801B
:100C60002D2D352D239F212DD22ECBB8001400140D
:100C70000014F5FEEBB80014001400140014EBB8D7
:100C800002E00A95F1F705E08BE290E06C2D4E2D25
:100C90002D2D0E940A01DD0C0150B1F70014CBB8D4
:100CA000001400140014D7FEEBB800140014001454
:100CB0000014EBB80014001400140014001483E0B6
:100CC00090E0680E791E8BE290E06C2D4E2D2D2D5C
:100CD0000E942B01E981FA811081252D129F112D8F
:100CE000CBB8001400140014D5FEEBB800140014A7
:100CF00000140014EBB800146A147B0408F463CFEA
:100D00001124E0908605F0908705009188051091E8
:100D10008905B401A3E0660F771FAA95E1F7680D76
:100D2000791D882777FD8095982F28EE33E040E0E5
:100D300050E00E94C913E20EF31E041F151FE0923B
:100D40008605F092870500938805109389057894AD
:100D50000E940C0EF10165837683878390870F9044
:100D60000F900F900F90CF91DF911F910F91FF90F7
:100D7000EF90DF90CF90BF90AF909F908F907F903B
:100D80006F905F903F902F9008951F93182F682FBA
:100D900062956F7060636A330CF0695D772767FD59
:100DA000709583E196E00E940911612F6F70606376
:100DB0006A330CF0695D772767FD709583E196E0F3
:100DC0000E9409111F910895EF92FF920F931F93B4
:100DD000CF93DF9383E196E00E949F10892B09F463
:100DE00083C081E080933A040E94FE0D2091630449
:100DF00030916404442737FD4095542F260F371F48
:100E0000481F591F20936D0430936E0440936F0464
:100E10005093700483E196E00E94D010182F8091C7
:100E20003B04882329F083E196E0612F0E94FE11A4
:100E3000812F80538A3058F5809165049091660423
:100E4000892B31F481E090E09093660480936504EF
:100E5000E0916504F0916604EE0FFF1FEB59FB4F24
:100E6000808191819C01A3E0220F331FAA95E1F7B5
:100E7000880F991F280F391F20533040812F992741
:100E800087FD9095280F391F318320832DC01C3298
:100E900001F5809165049091660482309105CCF44F
:100EA000892B31F481E090E090936604809365048F
:100EB000E0916504F09166043196F0936604E09346
:100EC00065043197EE0FFF1FE959FB4F1182108225
:100ED0000BC0812F0E941F021092660410926504BD
:100EE000109268041092670480913A04882309F0F4
:100EF000DDC0E0906D04F0906E0400916F041091DD
:100F000070040E94FE0D6E157F058007910708F49E
:100F1000CDC08091090190910A01FC01EE0FFF1FE5
:100F2000E80FF91F2AE431E0C90160E070E0AF0189
:100F30000E940315E0900F01F09010010091110143
:100F40001091120188EE93E0A0E0B0E0E80EF91EE7
:100F50000A1F1B1F0E94FE0DE616F7060807190759
:100F600020F48FE380934A0103C08FE380934C0108
:100F700085E00E945E0F892B29F480914C01815CF1
:100F800080934C0186E00E945E0F892B29F48091AA
:100F90004C01815C80934C0187E00E945E0F892B9D
:100FA00029F480914C01815C80934C0120916B0469
:100FB00030916C04237030702130310599F022306B
:100FC0003105F1F080910D0190910E01232B29F54F
:100FD000FC01EE0FFF1FE80FF91FE65BFE4F8FEFDE
:100FE000808326C080910D0190910E01FC01EE0FCF
:100FF000FF1FE80FF91FE65BFE4F8FEF818318C0DC
:1010000080910D0190910E01FC01EE0FFF1FE80F82
:10101000F91FE65BFE4F8FEF0AC0FC01EE0FFF1FCA
:10102000E80FF91FE65BFE4F8FEF80838183828399
:101030008091090190910A011816190654F4E09163
:101040003601F0913701CF01EE5BFF4F60810E94C6
:10105000CF0C80910D0190910E01019690930E019D
:1010600080930D012091090130910A0182179307A5
:101070007CF081E090E090930E0180930D018091CF
:101080006B0490916C04019690936C0480936B04B4
:101090000E94FE0D6E5C7F4F8F4F9F4F60936D04DB
:1010A00070936E0480936F04909370048091720427
:1010B000882309F459C080913C048823F1F1C0E0F1
:1010C000D0E011C0209729F083E196E06CE20E9405
:1010D000FE11E0913804F0913904EC0FFD1F80817E
:1010E0000E94C50621968091710490E0C817D90727
:1010F0004CF383E196E060E071E00E9472130EC051
:1011000080917104E0913804F0913904E80FF11DE9
:101110001082809171048F5F8093710480917104BB
:1011200090E04091090150910A019A01220F331F6A
:10113000240F351F821793071CF3809109019091AA
:101140000A011816190654F4E0913601F09137019E
:10115000CF01EE5BFF4F60810E94CF0C10927204B2
:1011600088E061E00E942B0F8091630490916404F9
:1011700018161906ACF480913A04882389F0E0909F
:101180006D04F0906E0400916F04109170040E9441
:10119000FE0D6E157F058007910710F010923A043E
:1011A000DF91CF911F910F91FF90EF90089581E013
:1011B0008093B804609395041092B6041092B7041B
:1011C00008952091940430E080919304281B310904
:1011D000C90108954091930480919404481718F030
:1011E0002FEF3FEF0AC0E42FF0E0ED58FB4F808176
:1011F000282F30E04F5F40939304C9010895E09198
:10120000930480919404E81718F0EFEFFFEF06C005
:10121000F0E0ED58FB4F8081E82FF0E0CF0108951A
:101220000895AC012091BB043091BC042115310517
:10123000E1F090919304809194049817B0F090E0BD
:1012400008C0FA01EA0FFB1F8081AD58BB4F8C9399
:101250009F5FA92FB0E0A617B7079CF310929304E5
:1012600060939404CB01F90109950895E091B904C4
:10127000F091BA04309729F01092B6041092B70496
:10128000099508951092C0041092BF0488EE93E06F
:10129000A0E0B0E08093C1049093C204A093C30483
:1012A000B093C4048AE291E09093BE048093BD049D
:1012B0000895CF92DF92EF92FF920F931F93CF93F7
:1012C000DF937C016B018A018091B8048823A1F02F
:1012D000C0E0D0E00DC0D701ED91FC91D601AC0F7C
:1012E000BD1F0190F081E02DC7016C9109952196F9
:1012F000C017D10780F304C0CB01642F0E94A60A57
:10130000C801DF91CF911F910F91FF90EF90DF9077
:10131000CF900895DF93CF930F92CDB7DEB7FC0146
:1013200069838091B8048823C9F08091B704803222
:1013300038F081E090E09383828320E030E015C0B4
:101340008091B604E82FF0E0EA56FB4F9981908334
:101350008F5F8093B6048093B70405C0CE010196D9
:1013600061E00E94A60A21E030E0C9010F90CF9110
:10137000DF9108950F93062F8091950466E974E03C
:101380004091B70421E00E94510A1092B6041092D5
:10139000B7041092B8040F91089561E00E94BA0951
:1013A0000895413208F040E2862F63E774E00E941E
:1013B000080A1092930480939404089521E00E94F7
:1013C000D109089510929304109294041092B604D7
:1013D0001092B7040E945C0C08950F931F938C0128
:1013E000862F0E94040A86E399E00E94C60A81E1E2
:1013F00099E00E94C10AC8010E94E2091F910F9161
:1014000008950E94ED090895880F8093BA00089509
:10141000382F413210F040E042C08091C904882347
:10142000E1F791E09093C9042093CB048FEF809370
:1014300036051092F10441504093F2044F5F9093AF
:10144000CA048091CA04330F832B8093CA0480910D
:10145000CC04813041F41092CC048091CA04809372
:10146000BB0085EC01C085EE8093BC008091C9046F
:101470008130E1F38091F104841710F44091F1047C
:1014800020E030E00AC0FB01E20FF31FD901AF52A8
:10149000BB4F8C9180832F5F3F4F2417A0F3842F85
:1014A00008950F931F93582F122F413210F081E0AF
:1014B0004AC08091C9048823E1F782E08093C9047F
:1014C0000093CB048FEF809336051092F104409384
:1014D000F204A1EDB4E0FB0102C081918D938E2F47
:1014E000861B8417D0F31092CA048091CA04550F4A
:1014F000852B8093CA048091CC04813041F41092F2
:10150000CC048091CA048093BB0085EC01C085EEB9
:101510008093BC00112321F08091C9048230E1F353
:10152000809136058F3F11F480E00DC08091360523
:10153000803211F482E007C080913605803311F0CB
:1015400084E001C083E01F910F910895482F61321C
:1015500010F081E008958091C904843011F082E098
:10156000089560931405A3EFB4E0842F9C01F90162
:1015700002C081918D938E2F841B8617D0F380E05B
:1015800008959093D0048093CF0408959093CE044F
:101590008093CD0408951F920F920FB60F921124DD
:1015A0002F933F934F935F936F937F938F939F936B
:1015B000AF93BF93EF93FF938091B90090E0887F42
:1015C00090708036910509F4F2C081369105CCF512
:1015D0008832910509F47BC089329105B4F48031D9
:1015E000910509F46FC0813191053CF4009709F42D
:1015F00047C1089709F04FC165C08831910509F4CA
:1016000066C0809709F047C182C08034910509F413
:10161000A4C08134910544F48033910509F482C05B
:10162000C89709F038C189C08035910509F489C08F
:101630008835910509F496C08834910509F02BC1CD
:10164000AEC08839910509F413C189399105ECF4CC
:101650008837910509F4ABC0893791054CF4883679
:10166000910509F4A4C08037910509F014C19FC009
:101670008838910509F4FCC08039910509F49DC0B2
:101680008038910509F007C198C0803B910509F4A5
:10169000C6C0813B91054CF4803A910509F49FC086
:1016A000883A910509F0F7C0BAC0803C910509F469
:1016B000E3C0883C910509F4DFC0883B910509F03F
:1016C000EAC0C2C08091CA048093BB00CFC0909191
:1016D000F1048091F204981768F49091F104E92FD5
:1016E000F0E0EF52FB4F80818093BB009F5F9093AF
:1016F000F104BCC08091CB04882309F44BC085ED74
:101700008093BC008091BC0084FDFCCFC2C080E20D
:101710008093360585ED8093BC008091BC0084FDEC
:10172000FCCFB7C080E38093360585ED8093BC0085
:101730008091BC0084FDFCCFACC088E3809336056B
:101740009BC08091F1049091BB00E82FF0E0EF5234
:10175000FB4F90838F5F8093F1049091F10480910F
:10176000F20482C08091F1049091BB00E82FF0E078
:10177000EF52FB4F90838F5F8093F1048091CB04F5
:10178000882341F085ED8093BC008091BC0084FDEE
:10179000FCCF7FC081E08093CC0484EA6EC085EDED
:1017A0008093BC008091BC0084FDFCCF72C083E0BC
:1017B0008093C9041092350559C080913505803257
:1017C00008F056C0809135059091BB00E82FF0E0FD
:1017D000EB5EFA4F90838F5F8093350547C0809111
:1017E0003505803230F4E0913505F0E0EB5EFA4FDC
:1017F000108285ED8093BC008091BC0084FDFCCFFD
:101800001092C90460913505E091CF04F091D004A5
:1018100085E195E070E00995109235052DC084E0D2
:101820008093C9041092130510921405E091CD0421
:10183000F091CE04099580911405882329F481E064
:10184000809314051092F30490911305E92FF0E0B2
:10185000ED50FB4F80818093BB009F5F90931305F9
:101860009091130580911405981710F485EC01C030
:1018700085E88093BC000FC085EC8093BC0009C054
:101880001092360585ED8093BC008091BC0084FDEC
:10189000FCCF1092C904FF91EF91BF91AF919F913E
:1018A0008F917F916F915F914F913F912F910F9009
:1018B0000FBE0F901F9018951092C90481E080937D
:1018C000CB041092CC0482E161E00E942B0F83E1F3
:1018D00061E00E942B0FE9EBF0E080818E7F808336
:1018E00080818D7F808388E48093B80085E4809335
:1018F000BC000895DF92EF92FF920F931F93CF9356
:10190000DF93EC017B01101611062CF0D22E032F71
:1019100020E030E002C0D02E012FC05CDF4FA88154
:10192000B981C054D040FE0160E070E007C0808102
:1019300091813896892B41F06F5F7F4F6A177B0743
:10194000B4F3EE24FF2422C0E3E0660F771FEA958C
:10195000E1F7DE01A60FB71F1196FC92EE92FE0191
:10196000E60FF71F5383428317963C932E931697E7
:10197000FB013496EC0FFD1FD0820183D701ED915E
:10198000FC910190F081E02DC7010995C701DF911D
:10199000CF911F910F91FF90EF90DF900895DF920C
:1019A000EF92FF920F931F93CF93DF93D62EEC010C
:1019B00000E010E050E4E52EF12CE80EF91E1DC009
:1019C000A881B9811097F9F0ED91FC9111972E81C2
:1019D0003F81C901880F991F820F931F6A817B8104
:1019E000680F791F4C815D810084F185E02DCD0168
:1019F0002D2D09950F5F1F4F2896F701808191814A
:101A000008171907ECF2DF91CF911F910F91FF900A
:101A1000EF90DF900895FC01E05CFF4F88E090E0DC
:101A2000819391938FEF8083E254F040CF0160E087
:101A300040E450E00E942E0D089587E395E00E9457
:101A40000B0D84E592E3A0EEB0E080937A059093CD
:101A50007B05A0937C05B0937D050895DC0140FFD4
:101A600003C001C06D936D934250E0F75040D0F732
:101A70000895823000F5E82FF0E0EE0FFF1FE258E6
:101A8000FA4F71836083882319F08130A1F408C074
:101A9000809169008C7F842B80936900E89A089577
:101AA00080916900440F551F440F551F837F842B7D
:101AB00080936900E99A08951F920F920FB60F92D2
:101AC00011242F933F934F935F936F937F938F9343
:101AD0009F93AF93BF93EF93FF9380917E05909177
:101AE0007F05892B29F0E0917E05F0917F0509950E
:101AF000FF91EF91BF91AF919F918F917F916F91E6
:101B00005F914F913F912F910F900FBE0F901F90BB
:101B100018951F920F920FB60F9211242F933F9397
:101B20004F935F936F937F938F939F93AF93BF93E5
:101B3000EF93FF938091800590918105892B29F087
:101B4000E0918005F09181050995FF91EF91BF919A
:101B5000AF919F918F917F916F915F914F913F9145
:101B60002F910F900FBE0F901F9018951F920F92FC
:101B70000FB60F9211242F933F938F939F93AF93A0
:101B8000BF938091860590918705A0918805B091BB
:101B9000890530918A050196A11DB11D232F2D5F66
:101BA0002D3720F02D570196A11DB11D20938A05D8
:101BB0008093860590938705A0938805B093890547
:101BC0008091820590918305A0918405B09185054F
:101BD0000196A11DB11D8093820590938305A0936A
:101BE0008405B0938505BF91AF919F918F913F91EF
:101BF0002F910F900FBE0F901F9018958FB7F894EC
:101C0000209186053091870540918805509189057E
:101C10008FBFB901CA0108959FB7F894209182053A
:101C200030918305409184055091850586B5A89B28
:101C300006C08F3F21F02F5F3F4F4F4F5F4F9FBF39
:101C4000542F432F322F2227280F311D411D511DA4
:101C500082E0220F331F441F551F8A95D1F7B90127
:101C6000CA010895EF92FF920F931F93CF93DF93D2
:101C70007B018C010E940C0EEB010EC00E940C0E29
:101C80006C1B7D0B685E7340C8F30894E108F10893
:101C900001091109C851DC4FE114F10401051105D6
:101CA00069F7DF91CF911F910F91FF90EF90089509
:101CB000019739F0880F991F880F991F0297019794
:101CC000F1F70895789484B5826084BD84B581600D
:101CD00084BD85B5826085BD85B5816085BDEEE634
:101CE000F0E0808181608083E1E8F0E01082808113
:101CF00082608083808181608083E0E8F0E0808181
:101D000081608083E1EBF0E0808184608083E0EBA0
:101D1000F0E0808181608083EAE7F0E08081846088
:101D200080838081826080838081816080838081E4
:101D3000806880831092C1000895982F8E3008F03B
:101D40009E509770809113018295880F880F807C38
:101D5000892B80937C0080917A00806480937A0044
:101D600080917A0086FDFCCF209178004091790027
:101D7000942F80E030E0282B392BC9010895CF93B0
:101D8000DF93482F50E0CA0182549F4FFC013491E9
:101D900046555F4FFA018491882369F190E0880FDE
:101DA000991FFC01E457FF4FA591B491FC01EA563D
:101DB000FF4FC591D491662351F42FB7F8948C91BD
:101DC000932F909589238C93888189230BC062304F
:101DD00061F42FB7F8948C91932F909589238C936D
:101DE0008881832B88832FBF06C09FB7F8948C917E
:101DF000832B8C939FBFDF91CF910895833071F037
:101E0000843028F48130A1F0823021F514C086306E
:101E1000B1F08730D1F08430E9F404C080918000C3
:101E20008F7703C0809180008F7D8093800008951C
:101E300084B58F7702C084B58F7D84BD089580916D
:101E4000B0008F778093B00008958091B0008F7DAF
:101E50008093B0000895FF920F931F93F62E482FA2
:101E600050E0CA018E529F4FFC012491CA01825456
:101E70009F4FFC01149146555F4FFA0104910023D6
:101E8000C9F0222319F0822F0E94FE0EE02FF0E00D
:101E9000EE0FFF1FEA56FF4FA591B4919FB7F8943C
:101EA000FF2021F48C911095812302C08C91812B0D
:101EB0008C939FBF1F910F91FF9008950F931F93D5
:101EC000482F50E0CA018E529F4FFC012491CA0155
:101ED00082549F4FFC01049146555F4FFA011491C3
:101EE000112319F420E030E015C0222319F0822FCD
:101EF0000E94FE0E812F90E0880F991F80569F4F01
:101F0000FC01A591B4918C9120E030E0802311F088
:101F100021E030E0C9011F910F91089508951F92AB
:101F20000F920FB60F9211242F933F934F938F93DD
:101F30009F93EF93FF938091C00082FD1DC040915D
:101F4000C6002091CB053091CC052F5F3F4F2F73FA
:101F500030708091CD059091CE052817390771F02A
:101F6000E091CB05F091CC05E557FA4F40833093D3
:101F7000CC052093CB0502C08091C600FF91EF9164
:101F80009F918F914F913F912F910F900FBE0F9086
:101F90001F901895E0911F06F0912006E05CFF4F1E
:101FA0008191919120813181821B930B8F7390706D
:101FB000892B11F00E948E0F08951F920F920FB679
:101FC0000F9211242F933F938F939F93EF93FF933F
:101FD00020910F0630911006809111069091120603
:101FE0002817390731F48091C1008F7D8093C1009B
:101FF00014C0E0911106F0911206E153FA4F2081CE
:10200000809111069091120601968F7390709093B3
:102010001206809311062093C600FF91EF919F91C5
:102020008F913F912F910F900FBE0F901F90189599
:10203000AF92BF92DF92EF92FF920F931F93CF93D5
:10204000DF93EC017A018B01DD24403081EE5807EB
:1020500080E0680780E0780711F0DD24D39491E0F8
:10206000A92EB12CEC89FD89DD2069F0C50108A0FD
:1020700002C0880F991F0A94E2F7808360E079E03C
:102080008DE390E005C0108260E874E88EE190E096
:10209000A80197010E94A7132150304040405040B2
:1020A000569547953795279580E12030380720F0E1
:1020B000DD2011F0DD24D6CFE889F9893083EA8963
:1020C000FB89208319A2EE89FF89408121E030E05D
:1020D000C9010C8C02C0880F991F0A94E2F7482BA3
:1020E0004083EE89FF894081C9010D8C02C0880FB1
:1020F000991F0A94E2F7482B4083EE89FF894081BB
:10210000C9010E8C02C0880F991F0A94E2F7482B70
:102110004083EE89FF8980810F8C02C0220F331F1C
:102120000A94E2F7209528232083DF91CF911F9115
:102130000F91FF90EF90DF90BF90AF900895DC017A
:102140001C96ED91FC911D97E05CFF4F2191319120
:1021500080819181281B390B2F733070C90108953C
:10216000DC011C96ED91FC911D97E05CFF4F2081F6
:102170003181E054F040DF01AE5BBF4F8D919C9107
:1021800011972817390719F42FEF3FEF07C08D91EA
:102190009C91E80FF91F8081282F30E0C901089534
:1021A000DC011C96ED91FC911D97E05CFF4F2081B6
:1021B0003181E054F040DF01AE5BBF4F8D919C91C7
:1021C00011972817390719F42FEF3FEF10C08D91A1
:1021D0009C911197E80FF91F20818D919C91119787
:1021E00001968F73907011969C938E9330E0C90185
:1021F0000895DC0191968C919197882339F054963B
:10220000ED91FC915597808186FFF9CF91961C92B4
:102210000895CF93DF93EC01EE85FF85E05CFF4FDF
:1022200020813181E054F0402F5F3F4F2F73307099
:10223000DF01AE5BBF4F8D919C9111972817390735
:10224000D1F3E05CFF4F80819181E054F040E80FD2
:10225000F91F6083EE85FF85E05CFF4F31832083AB
:10226000EE89FF89208181E090E00F8C02C0880F09
:10227000991F0A94E2F7282B208381E089A3EC8937
:10228000FD8980818064808381E090E0DF91CF913F
:102290000895109216061092150688EE93E0A0E0BD
:1022A000B0E08093170690931806A0931906B09398
:1022B0001A068EE391E090931406809313068BE840
:1022C00095E09093200680931F068FEC95E0909305
:1022D00022068093210685EC90E09093240680935B
:1022E000230684EC90E0909326068093250680ECEC
:1022F00090E0909328068093270681EC90E09093DD
:102300002A068093290682EC90E090932C06809315
:102310002B0686EC90E090932E0680932D0684E0A9
:1023200080932F0683E08093300687E08093310608
:1023300085E08093320681E0809333060895CF9341
:10234000DF930E94620E0E94C503CAECDFE00E9488
:10235000E4062097E1F30E94CA0FF9CF0E94FE1312
:102360000895CF92DF92EF92FF920F931F93CF9336
:10237000DF937C016B018A01C0E0D0E00FC0D60181
:102380006D916D01D701ED91FC910190F081E02DEF
:10239000C7010995C80FD91F01501040011511053B
:1023A00071F7CE01DF91CF911F910F91FF90EF90C8
:1023B000DF90CF900895EF92FF920F931F93CF93EA
:1023C000DF937C018B01C0E0D0E0F8010F5F1F4F6D
:1023D0006491662359F0D701ED91FC910190F08151
:1023E000E02DC7010995C80FD91FEFCFCE01DF91AE
:1023F000CF911F910F91FF90EF900895DC01ED9127
:10240000FC910190F081E02D09950895EF92FF92E3
:102410000F931F938C01DC01ED91FC910190F081F1
:10242000E02D6DE009957C01D801ED91FC910190C2
:10243000F081E02DC8016AE009959C012E0D3F1D39
:10244000C9011F910F91FF90EF900895EF92FF92B5
:102450000F931F937C010E94DB118C01C7010E9426
:1024600006129C01200F311FC9011F910F91FF908F
:10247000EF900895EF92FF920F931F937C01DC0180
:10248000ED91FC910190F081E02D09958C01C7013F
:102490000E940612080F191FC8011F910F91FF908B
:1024A000EF900895CF93DF93EC016115710519F456
:1024B00020E030E00FC0DB010D900020E9F711971C
:1024C000A61BB70BE881F9810280F381E02DAD01F5
:1024D00009959C01C901DF91CF9108954F925F92B8
:1024E0007F928F929F92AF92BF92CF92DF92EF92A4
:1024F000FF920F931F93DF93CF93CDB7DEB7A197D2
:102500000FB6F894DEBF0FBECDBF2C01742ECB01E9
:10251000223008F42AE019A231E2C32ED12CCC0ECD
:10252000DD1E822E9924AA24BB24672D752FA501B8
:1025300094010E94A71379018A01C801B701A5017E
:1025400094010E947513472D461B0894C108D108B9
:102550004A3014F4405D01C0495CF6014083E11447
:10256000F1040105110521F07E2C5F2DC801DDCF9E
:10257000C201B6010E945212A1960FB6F894DEBFB6
:102580000FBECDBFCF91DF911F910F91FF90EF90C4
:10259000DF90CF90BF90AF909F908F907F905F9093
:1025A0004F900895DC012115310541F4ED91FC9126
:1025B0000190F081E02D642F099508950E946E121C
:1025C0000895CF92DF92EF92FF920F931F936C01C9
:1025D000E62E9A01FF2400E010E0B801A7010E9456
:1025E000D2128C01C6010E940612080F191FC801E1
:1025F0001F910F91FF90EF90DF90CF900895CF92B1
:10260000DF92EF92FF920F931F93CF93DF93EC0132
:102610006A017B012115310541F4E881F9810190BE
:10262000F081E02D642F09951FC02A303105D1F4C7
:1026300077FF17C0E881F9810190F081E02D6DE20C
:1026400009958C0144275527BA014C195D096E097B
:102650007F09CE012AE00E946E129801280F391FCF
:1026600004C02AE00E946E129C01C901DF91CF9143
:102670001F910F91FF90EF90DF90CF900895EF9210
:10268000FF920F931F937C010E94FF128C01C701E0
:102690000E9406129C01200F311FC9011F910F914A
:1026A000FF90EF900895CF92DF92EF92FF920F93F9
:1026B0001F936C017B019A010027F7FC0095102FF6
:1026C000B801A7010E94FF128C01C6010E940612E8
:1026D000080F191FC8011F910F91FF90EF90DF9015
:1026E000CF9008950E9452120895629FD001739F67
:1026F000F001829FE00DF11D649FE00DF11D929F9E
:10270000F00D839FF00D749FF00D659FF00D9927DC
:10271000729FB00DE11DF91F639FB00DE11DF91F00
:10272000BD01CF011124089597FB092E07260AD079
:1027300077FD04D049D006D000201AF47095619539
:102740007F4F0895F6F7909581959F4F0895A1E2E8
:102750001A2EAA1BBB1BFD010DC0AA1FBB1FEE1F1B
:10276000FF1FA217B307E407F50720F0A21BB30B66
:10277000E40BF50B661F771F881F991F1A9469F7E2
:1027800060957095809590959B01AC01BD01CF013E
:10279000089597FB092E05260ED057FD04D0D7DFEC
:1027A0000AD0001C38F450954095309521953F4F44
:1027B0004F4F5F4F0895F6F790958095709561950E
:1027C0007F4F8F4F9F4F0895AA1BBB1B51E107C03E
:1027D000AA1FBB1FA617B70710F0A61BB70B881FB1
:1027E000991F5A95A9F780959095BC01CD01089540
:1027F000EE0FFF1F0590F491E02D0994CF93DF9326
:10280000BC018230910510F462E070E0A0913706BF
:10281000B0913806ED01E0E0F0E040E050E021C08A
:10282000888199818617970769F48A819B813097FF
:1028300019F09383828304C09093380680933706FF
:10284000FE0134C06817790738F44115510519F0B5
:102850008417950708F4AC01FE018A819B819C01D5
:10286000E9012097E9F641155105A9F1CA01861B36
:10287000970B049708F4BA01E0E0F0E02AC08D91CC
:102880009C91119784179507F9F46417750781F4E3
:1028900012968D919C911397309719F093838283B0
:1028A00004C09093380680933706FD0132964FC0DE
:1028B000CA01861B970BFD01E80FF91F6193719305
:1028C00002978D939C9343C0FD01828193819C016B
:1028D000D9011097A1F68091350690913606892B83
:1028E00041F4809105019091060190933606809302
:1028F000350640910701509108014115510541F4F9
:102900004DB75EB78091030190910401481B590BAC
:10291000209135063091360624173507B0F4CA01E8
:10292000821B930B8617970780F0AB014E5F5F4FBA
:102930008417950750F0420F531F5093360640936B
:102940003506F9016193719302C0E0E0F0E0CF0138
:10295000DF91CF910895CF93DF93009709F450C092
:10296000EC0122971B821A82A0913706B09138069B
:10297000109709F140E050E0AC17BD0708F1BB83A8
:10298000AA83FE0121913191E20FF31FAE17BF0719
:1029900079F48D919C911197280F391F2E5F3F4F2D
:1029A0003983288312968D919C9113979B838A83F8
:1029B0004115510571F4D0933806C093370620C0F5
:1029C00012968D919C911397AD01009711F0DC0147
:1029D000D3CFFA01D383C28321913191E20FF31F48
:1029E000CE17DF0769F488819981280F391F2E5F80
:1029F0003F4FFA01318320838A819B8193838283B5
:102A0000DF91CF910895DC0101C06D93415050409A
:082A1000E0F70895F894FFCFF0
:102A18000D0A0020003906000032002000010018CD
:102A2800FCFFFF0100000000E600A100EF00A80580
:102A3800A604A900AB00000000008A095909E108B2
:102A4800EA08FF08100937053705000000000911DA
:0A2A5800B1119F10D010B010F9105A
:00000001FF
